:0A00060000308A001C28000043307F
:100010008400000803191B280130F800F701F70BD2
:100020000F28F80B0E284A30F700F70B15280000B0
:100030000000800B0C28003484011F3083058316D8
:100040001F08C0399F009B01073083129F001930A1
:100050008316990026309800903083129800413022
:10006000A1004330A2004130A3004530A400A50107
:100070004630A6003930A700A8014130A90044301D
:10008000AA00AB018316850183128501FF30831618
:100090008600831298172C3084008403840A8C1EF7
:1000A0004F281A0880000D300002031D4E288001E1
:1000B000981383168601831221083702031D6428D2
:1000C000220838020319051423083702031D6C287F
:1000D000240838020319051426083702031D742862
:1000E000270838020319851429083702031D7C28C4
:1000F0002A083802031905150430C200FA30C3007B
:100100000720C20B7E280430C200FA30C30007204B
:10011000C20B85288501181218161A08C0001A0883
:0A012000C0001A08C0004628630062
:040000008A01032846
:00000001FF
